:0300000002000EED
:0300030002019F58
:20000B0002019675811AD2AFD2A91201A280FE12001B80FBC82581C822C92581C97A002229
:20002B00D083D082CF2581F581CFC082C08322CF2581F581CF22FBE493CB22FCE493FB7492
:20004B000193CC22FAE493F9740193CA2229F9E5F03AFA227C00CB30E7011CCB2275F0009B
:20006B0030E70215F022FDE493FF7401934F7004A3A3800C740293B50510740393B5F00A99
:20008B00E493C0E0740193C0E022A3A3A3A380D7FEEBA4FD8EF0ECA4FCEB8EF0A4C5F02C0F
:2000AB002DC5F02211B58EF0ED22C002C001AAF0F97E007D007F11C3E933F9EA33FADF0867
:2000CB00F5F0E9D001D00222ED33FDEE33FEC3ED9BF5F0EE9C40E0ADF0FED380DBBB0001E7
:2000EB0022C333C5F033C5F0DBF722BB000122C3C5F013C5F013DBF722240280022401C595
:20010B00F03400C5F022C394028003C39401C5F09400C5F0223116F4C5F0F4C5F02245F095
:20012B007022042231784024801A3178401E7014801A3178400E7014800A3178500E8004A0
:20014B00318C6008E4F5F022318C60F8E4F5F00422318C40F780ED318C40F170E780ED313C
:20016B008C40E170E780DD318C50E180D7C39BC5F09C20E70720D207C345F02220D2F9D340
:20018B0022C5F0C39C7003E5F09B22758CDC758A000508320508327400F508740075F00075
:2001AB00F50985F00A740075F000F51585F016748075F025C0E0C0F0120CA115811581127E
:2001CB000CF0795D7A0DE98AF0F9AAF089828A83E493A3F5F0E493C5F0C0E0C0F0120CC450
:2001EB0015811581120369740175F00045F07003020237E5081200687B0112005F12012FF7
:20020B0045F060030201FE7400F5081202FD12038C1209071203C61204671205581206C650
:20022B00120743120927120A140201F2227F0912002B740078FC12001FF6740075F0000819
:20024B00F608A6F078FC12001FE61200687B0A12005F12015345F070030202AF801678FD38
:20026B0012001FE60886F012010818F608A6F012011680D0741175F000C0E0C0F0120CD86E
:20028B0015811581120CF078FC12001FF608E60886F079F612002412005878FC12001FE678
:2002AB00F702026978FD12001FE60886F079F61200241200587400F778FD12001FE6088631
:2002CB00F07B007C0012014B45F070030202E274FF75F0FF0202F879F6120024E98AF0C0A5
:2002EB00E0C0F0120D07158115810202F87FF702003AE59854011200687B0012005F120118
:20030B005345F0700302031B120CF0F51002031F74FFF51022E59854011200687B0012000D
:20032B005F12015345F0700302033E120D52F51002034274FFF5102279617A0DE98AF0F9EE
:20034B00AAF089828A83E493A3F5F0E493C5F0C0E0C0F0120CC41581158112036922795FDF
:20036B007A0DE98AF0F9AAF089828A83E493A3F5F0E493C5F0C0E0C0F0120CC41581158154
:20038B0022E5101200687B0A12005F12014B45F070030203C5795D7A0DE98AF0F9AAF0891F
:2003AB00828A83E493A3F5F0E493C5F0C0E0C0F0120CC41581158112036922E5101200680B
:2003CB007B6512005F12014B45F07003020466D2B3D2B4C2B5C2B6C2B7120B03C2B374646F
:2003EB0075F000C0E0C0F0120AB115811581740075F000F50985F00AE509850AF07B017C89
:20040B000012012F45F070030204518012E509850AF0120108F50985F00A12011680D9C2B5
:20042B00A7740A75F000C0E0C0F0120AB115811581D2A7740A75F000C0E0C0F0120AB11550
:20044B00811581020418D2B3746475F000C0E0C0F0120AB11581158112034322E5101200D0
:20046B00687B7712005F12014B45F07003020557D2B3C2B4D2B5D2B6D2B7D2A7120B03E531
:20048B000F75F0007BFF7C0012014B45F0700302049FC2B3746475F000C0E0C0F0120AB16D
:2004AB0015811581740075F000F51385F014740075F000F50985F00AE509850AF0AB15AC6C
:2004CB001612015C45F070030205428012E509850AF0120108F50985F00A12011680D9740E
:2004EB001175F000C0E0C0F0120CD815811581E509850AF0F51185F012851190E51244802E
:20050B00F5A0120B03120D52F580741375F000C0E0C0F0120CD815811581E5138514F02531
:20052B0080C5F03400C5F0F51385F014120A600030B2FD000204D8D2B3746475F000C0E066
:20054B00C0F0120AB1158115811203432205810581E5101200687B7212005F12014B45F001
:20056B007003020613740075F000F51385F014D2B3D2A7C2B4D2B5D2B6D2B77431F50D7451
:20058B000075F00078FD12001FF608A6F078FD12001FE60886F0AB15AC1612015C45F07011
:2005AB0003020610801678FD12001FE60886F012010818F608A6F012011680D178FD1200AD
:2005CB001FE60886F0F51185F012851190E5124480F5A0C2B5120B037580FFE5138514F07E
:2005EB002580C5F03400C5F0F51385F014E580120068C0E0C0F012061815811581D2B512F8
:20060B00063F0205B1120343158115812278FB12001FE6F50BE50B75F0007B047C00120040
:20062B00F6F50B12066278FB12001FE6540FF50B120662221203207B137C0012014B45F0E4
:20064B0070030206611203207B117C0012015345F0600302065022E50B75F0007B097C00A9
:20066B0012016A45F0700302068AE50B243775F000C0E0C0F0120CD81581158102069CE50D
:20068B000B243075F000C0E0C0F0120CD81581158122E5801200687BFF12005F1201534582
:2006AB00F070030206C57430F50DE519851AF0120108F51985F01A12011622E5101200685A
:2006CB007B6C12005F12014B45F07003020742C2B3D2A7D2B4D2B5D2B6D2B7746475F0001D
:2006EB00C0E0C0F0120AB115811581120A60740575F000C0E0C0F0120AB115811581C2B68B
:20070B00C2B7120B03120A60740575F000C0E0C0F0120AB115811581C2B5D2B6C2B7120BFD
:20072B0003120A60740575F000C0E0C0F0120AB11581158112034322E5101200687B63122F
:20074B00005F12014B45F07003020787749975F00DC0E0C0F0E5138514F01201222401C52A
:20076B00F03400C5F0C0E0C0F0740275F000120B4C158115811581158112034322D2B3D2D8
:20078B00A7C2B4D2B5C2B6C2B7743175F000F51185F012851190E5124480F5A0C2B5120B18
:2007AB00037580FFE580F50ED2B5E5118512F0120108F51185F012120116851190E5124499
:2007CB0080F5A0C2B5120B037580FFE580F50F2205810581120788E50E75F00090084802FC
:2007EB000071740075F010F51785F018020868740075F010F51785F018020868740075F0BC
:20080B0020F51785F018020868740075F020F51785F018020868740075F050F51785F018DC
:20082B00020868740075F050F51785F018020868740075F000F51785F0180208683B08FFE1
:20084B00002E086500210855001408620007085200FA076100ED0751000000680874007595
:20086B00F000F51385F014740075F000F51985F01AD2B3D2A7C2B4D2B5D2B6D2B77431F5D0
:20088B000D740075F00078FD12001FF608A6F078FD12001FE60886F0AB17AC1812015C45E9
:2008AB00F07003020902801678FD12001FE60886F012010818F608A6F012011680D178FD67
:2008CB0012001FE60886F0F51185F012851190E5124480F5A0C2B5120B037580FFE513856D
:2008EB0014F02580C5F03400C5F0F51385F01412069DD2B50208B31581158122E5101200C7
:20090B00687B7312005F12014B45F07003020926120238F51585F01612034322E51012006C
:20092B00687B6712005F12014B45F07003020A131207DBE50E75F0007BFF7C0012015345DF
:20094B00F07003020A0074A975F00DC0E0C0F0E50E75F000C0E0C0F0740275F000120B4C52
:20096B001581158115811581E50F75F0007BFF7C0012014B45F0700302099674B875F00D80
:20098B00C0E0C0F0120CC415811581E50F75F0007B057C0012014B45F070030209B974BD9E
:2009AB0075F00DC0E0C0F0120CC41581158174C175F00DC0E0C0F0E519851AF0C0E0C0F088
:2009CB00740275F000120B4C158115811581158174D575F00DC0E0C0F0E5158516F0C0E040
:2009EB00C0F0740275F000120B4C1581158115811581020A1074E875F00DC0E0C0F0120C48
:200A0B00C41581158112034322E5101200687B7012005F12014B45F07003020A5F1207DB31
:200A2B0074FA75F00DC0E0C0F0E50E75F000C0E0C0F0E519851AF0C0E0C0F0E5158516F071
:200A4B00C0E0C0F0740475F000120B4C7FF812002B12034322C2A7000000D2A72205810538
:200A6B0081740075F00078FD12001FF608A6F078FD12001FE60886F07B087C0012012F4547
:200A8B00F07003020AAC801678FD12001FE60886F012010818F608A6F012011680D1020A43
:200AAB0093158115812205810581740075F00078FD12001FF608A6F078FD12001FE6088611
:200ACB00F078F912001F860308860412012F45F07003020AFE801678FD12001FE60886F0CA
:200AEB0012010818F608A6F012011680CB120A68020AE2158115812205810581740075F00B
:200B0B000078FD12001FF608A6F078FD12001FE60886F07B017C0012012F45F07003020B97
:200B2B0047801678FD12001FE60886F012010818F608A6F012011680D1020B2E158115811B
:200B4B002223F42581F8868208868308E4FEFF93700122B42555A3E493B42D06430780A3EF
:200B6B00E493B4300343074024D0B40A00500CCE75F00AA42EFEA3E49380EDE493B464133E
:200B8B00E60886F030F708430720120120A6F018F68003B4750543070A801CB4780543075A
:200BAB00108014B46F0B430708800C120CDEA3809BB462624307027A00C004C005C006C073
:200BCB0007AB0753031F7C00E60886F01200B5A6F018F6EDD007D006D005D0042430B43A0C
:200BEB000040022407C0E00AE645F070CCA902EF30E506742D120CDE0A120C82D0E0120CB2
:200C0B00DED9F90808EF30E7A5EAC39E50A07420120CDE0A80F3B4630BAA01120C82E612B1
:200C2B000CDE80DFB4732BC082C08386820886837A00E4936004A30A80F8868318868212BB
:200C4B000C82E493A36005120CDE80F6D083D08280B1B4691986017A00E76004090A80F926
:200C6B00120C828601E7609B120CDE0980F7F97A01120C82E980A8EE601B8FF020F716C0EA
:200C8B0002EAC39E500D742030F6027430120CDE0A80EED0022278FB12001F860308860418
:200CAB00748075F0701200B5120120758921F58DF58B7588597598522278FB12001F8682C2
:200CCB00088683E4936034120CDEA380F678FB12001FE63099FDC299F599B40A1E740D80C2
:200CEB00F2E43098133098FDC298E5993099FDC299F599B40D02740A75F0002278FB12009F
:200D0B001F8601E4FBFCFFE709B42D030FE709C39430B40A005012FA740A75F00012009B44
:200D2B002AFBE5F03400FC80E4EB8CF0DF030201202278FB12001FE63099FDC299F5992231
:200D4B0074FFF5F030980A3098FDC298E59975F00022630D900D940D0A20456173792D445F
:200D6B006F776E6C6F616465722056322E3020666F722041544D454C2038394335312F35FF
:200D8B00322F3535000A203E000A206F6B000A2043484B53554D203D2025303478000A2074
:200DAB00666F756E6420383943253278002D313256002D3556000A206E6F6E626C616E6B4E
:200DCB00202575206279746573000A20627974657320636F756E746572202575000A204E64
:180DEB006F7420666F756E642038394378780025782C25752C257500E4
:00000001FF
